:030000000219FDE5
:03000B000200AA46
:03002B0002015C73
:03005B000202EEB0
:030073000202DBAB
:1000800002030406080C10182030406080040608A3
:100090000C10182030406080A0C00003070F1F0D17
:1000A0000D0403060D0503030202C2AFC0D0C0E079
:1000B000206214E5256009E473E525F4F58AD2622F
:1000C000D0E0D0D0D2AF3285268AC262E526F46075
:1000D0002F30682520720DD0E0D0D0C293C295C2D7
:1000E00097D2AF32C293C295C297206F0C20650998
:1000F000740AD5E0FDE57B4290D0E0D0D0D2AF329B
:10010000758A00C28DD26201F901B9306805206597
:1001100002D29301B9306805206502D29501B93049
:100120006805206502D29701B9C29230680A20653D
:10013000077408D5E0FDD29301B9C29430680A2053
:1001400065077408D5E0FDD29501B9C29630680AFA
:100150002065077408D5E0FDD29701B9C2AFC2ADE2
:1001600053E6EFC0D0C0E0D2D3D2AFC2CEE52A6012
:100170000720744F152A21C37800790020742EE5DA
:1001800080307E01F430E30278FF53DACF207E0323
:1001900043DA20307E0343DA10C2D8C271E58030E2
:1001A0007E01F430E30279FFC3E89970CB3061033C
:1001B000752A40207403752A40885CD270E8600379
:1001C000755F0020740DE52B6004152B21D343DAF5
:1001D00001C2D820700221E6A85C206102C2702012
:1001E000740221E488227882B6040385222420CF79
:1001F0000AD0E0D0D043E610D2AD32C2CF053A7873
:1002000002E52A6005307402152AC3E55C940140BA
:1002100005755F004127756000756900E55F240181
:10022000F55F5003755FFF7982B7020D306E1DC315
:10023000E52294324016854C227982B7030E306E47
:100240000BC3E52294324004798E8722C3E52395BF
:1002500022600840041523415B0523D8CA0569E5DF
:100260006970021569D56A69756A017808E56B607D
:10027000497805C3E569956B4057C3E569956C50AE
:10028000087801756A03020295C3E569956D50050A
:100290007801756A01C3E5629524401E7982B7042E
:1002A0000241C6206E14852462E569046003856BF3
:1002B00069756A0175233C0202D1E5622850057513
:1002C00062FF41C6F562E5620470067560FF7569FC
:1002D000FFD0E0D0D043E610D2AD32C2AF53E67FBC
:1002E0007592FA7593FFC260759104D2AF32C2AFB6
:1002F00053E6EFC2ADC0D0C0E0C0F0D2D3D2AFA8B9
:10030000FBA9FCC2D8307102615553DACF207E03BD
:1003100043DA10307E0343DA20D271E580307E016B
:10032000F420E302612C88278928A13A53DACF20F0
:100330007E0343DA20307E0343DA10C2D8C2713024
:100340007402A1267800E580307E01F430E302A13A
:1003500026885CA10E53DACF207E0343DA20307E5C
:100360000343DA10C271206102812E53DACF207E5E
:100370000343DA10307E0343DA20C2D8D2718857A3
:100380008958C3E89555F8E99556F97B007E087AB7
:1003900000C3E8948CE994005005755B00812088C7
:1003A0002178A2E6A8216055C3E894C8E9940050DA
:1003B00008E4D2E4FB7A0A61FBC3E89468E994019B
:1003C0005008E4D2E3FB7A0F61FBC3E894D0E994D0
:1003D000025008E4D2E2FB7A1E61FBC3E894A0E974
:1003E00094055008E4D2E1FB7A3C61FBC3E89498A1
:1003F000E994085008E4D2E0FB7A787E00C3E895DF
:1004000059FCE9955AFD30E70AECF42401FCEDF4BF
:100410003400FD755B00C3EC9AED9E5003755B01E3
:100420008859895A8557558558567802A10EC3E8D0
:100430009527F8E99528F9307C0281F2307B02811A
:10044000F2307A0281EB2075028151E9FDE8FC81EE
:1004500070E9C313F9E813F830790281EBE9C313AB
:10046000F9E813F830780281EBE9C313FDE813FCD7
:0F04700020612CC3EC941CED940240028187EDB7
:10047F00701EC3EC94C850180529E5297002152980
:10048F00C3E529940A5002A126755C00D270A126FB
:10049F00E529600215297400207F037896E624FA77
:1004AF00FEE43400FFC3EC9EFCED9FFD5006780088
:1004BF00790081F2C3EC94FFED9400400678FF7948
:1004CF000081F2EC8572F0A4C5F0A2F733F8790041
:1004DF00400302050E78FF790002050EE9C313F9F8
:1004EF00E813F8307C0EE9600278FFC3E81338F8A0
:1004FF00E43400F9C3E894FFE99400400278FF88E0
:10050F005CD270206102A126741FF4552F4BF52F7A
:10051F00C274EB7002D274752A40307403752A0AC4
:10052F00306102A13A20740353DAFE207403752B55
:10053F0020D0F0D0E0D0D0D2AD43E6103279010216
:10054F00056A790302056A790A02056A791E0205AE
:10055F006A796402056A79C802056A7817E4D5E0FA
:10056F00FDD8FAD9F6227A147B780205917A107B9E
:10057F008C0205917A0D7BB40205917A0B7BC80230
:10058F000591E573D5E001227902E4C294D5E0FD2F
:10059F00D295D5E0FDC295D5E0FDD294D5E0FDE929
:1005AF0020E002D29330E002D297E573D5E0FDE967
:1005BF0020E002C29330E002C2977496D5E0FDD9D5
:1005CF00C9EAF8D5E0FDD8FBDBB8C29422C37C00A2
:1005DF007D0075F00005F0EA33FAEB33FB50F6EBD4
:1005EF0013FBEA13FAC3E9FFE8FEE89AF8E99BF96F
:1005FF005004EFF9EEF8B3EC33FCED33FDD5F0DF3B
:10060F00EDF9ECF822E889F08A20D2D4F8A9F07B32
:10061F000030F70B7BFFF42401F8E9F43400F9E81C
:10062F008520F0A4ADF0F8E98520F0A4AFF0FEED41
:10063F002EF974003FFA7C04C3EA13FAE913F9E8C0
:10064F0013F8DCF48BF030F70AE8F42401F8E9F43E
:10065F003400F9E889F0C2D4F8A9F0227882B60400
:10066F000302070AC3E55C9419401EE52D5406707A
:10067F0018206E3678057994E7146007780A1460AD
:10068F00027812C3E54198401F306E098564627588
:10069F0069FF756A01852224E4F544F545F546F5B1
:1006AF0047F548C26E02070AD26E7994E7147013A9
:1006BF00E523F43333F913F8E9540104F9E854FE50
:1006CF000206FEE714147014E523F4333333F913E1
:1006DF00F8E9540304F9E854FC020706E523F43360
:1006EF00333333F913F8E954070404F9E854F8C322
:1006FF009440F8E99400F98844894522C3E54113F1
:10070F00F9E54013F8C3E54498F8E54599F9500C1D
:10071F00C3E89480E994FF4016020742C3E8947F30
:10072F00E994005003020742787F7900020742786C
:10073F008079FF8849894A22E5492546F8E54A35F7
:10074F0047F9854A20E4300701F43548FA30E709C4
:10075F00C3EA94F04015020780C3EA940F500302D6
:10076F00078078FF79FF7A0F020780780079007A87
:10077F00F0C3E5249561500AC374019524500B0210
:10078F00079EE54A20E70E02079EE54A30E70688F6
:10079F004689478A482278A5E6FAC3E54933F8E542
:1007AF004A33F9D114E930E70BC3E89480E994FF99
:1007BF004013E1D8C3E8947FE994005002E1D87860
:1007CF007F7900E1D8788079FFE820E715C3E5232A
:1007DF0098F84009C3E8940140030207FF7801022B
:1007EF0007FFE8F424012523F840030207FF78FFF1
:1007FF00884B2278A6E6FAA847A948120614E930D2
:10080F00E70CC3E89401E994FF4016020834C3E8EB
:10081F0094FFE99400500302083478FF790002082E
:10082F0034780179FFE920E715C3E54B98F84009C3
:10083F00C3E89401400302085B780102085BE8F407
:10084F002401254BF8400302085B78FF88242278A7
:10085F00FF20692879A1E76023E541601F74FF85B8
:0E086F0041F0848539F0306A0375F005A4F875
:10087D00C5F0600278FFC3E895645002A8648863F0
:10088D0022C3E5409440E5419401E5635003140112
:10089D009F046002F563227883E6F520120F3C7504
:1008AD00E89012054C75E89030EDFDA8BDA9BE127B
:1008BD000FE3756E55756F00C3740013FD745560AD
:1008CD006613FC74552CFC74003DFDECFAEDFBC376
:1008DD00E89AE99B4014E56E2455F56EE56F3400FA
:1008ED00F56FEA2CFAEB3DFB80E5AE6EAF6FC3E51D
:1008FD006F13F9E56E13F8C3E913F9E813F87A03EA
:10090D00C3E913F9E813F8DAF7AA201A7009756E1E
:10091D0000756F000209341AEA6008EE28FEEF39FF
:10092D00FFDAF88E6E8F6F2275E890227883E6FFDE
:10093D0030EDF9A8BDA9BE0570C3E570940840520D
:10094D00757000E9FA79A0E76044EA7007E5716017
:10095D001B02096DC3E895716010E5715006600CBE
:10096D00140209790460F9020979E571F571C394EE
:10097D00A8401B7561C0C394054013756180C39475
:10098D0005400B756140C39405400375610075BB4F
:10099D000122EFC39401601F7455601BC3E894FFDF
:1009AD00E994035012C3E8956EE9956F5009E5611E
:1009BD00600C15610209CBE561F460020561A86167
:1009CD00C3E524985002A824C3E89562400AA862A2
:1009DD00E562F4600385626188258826E570B407B9
:1009ED000375BB1E22743279A787F0A4C5F0A2F758
:1009FD0033F8C3E895614002A861882288248825D0
:100A0D0088268864227540007541F022C2AF75C8F2
:100A1D0020A8CCA9CDAA3A30CF010A75C824D2AFEF
:100A2D00AB3BAC3C883B893CC3E89BF8E99C206917
:100A3D0008F9306602612A4184AD3D8A3DF9EA9D8F
:100A4D00FA600678FF79FF4169AE3EAF3F8B3E8C71
:100A5D003FA83BA93CC3E89EF8E99FF9C3E54113C4
:100A6D00FBE54013FAE82AF540E93BF541500675E0
:100A7D0040FF7541FF41D1AA40AB41AC40AD417E35
:100A8D00047F02C3EB9404400D1E1FC3EB9408407A
:100A9D0005206A021E1FC3ED13FDEC13FCDEF7C328
:100AAD00EA9CFAEB9DFBEF6009C3E913F9E813F833
:100ABD00DFF7EA28FAEB39FB8A408B4150067BFFC2
:100ACD008B408B41C3EB94025002D2663069047F98
:100ADD000341FC7892E6FFC3E537948240110FC3C2
:100AED00E53794A040010FC3EF940640027F057EC9
:100AFD0002E541C4540FF9E541C454F0F8E540C492
:100B0D00540F28F8C3E89EFAE99400FB4009C3EAA4
:100B1D009402EB940050047A02E4FB6176AA40AB98
:100B2D0041EBC4FEEAC4540F4EFCC3EA9CFAEB94AD
:100B3D0000FBC3E813C313F8EA28FAEB3400FB8A71
:100B4D00408B41C3EB94024002C2667802EBC4FEB7
:100B5D007B00EAC4540F4EFAC3EA98FA4005C394D9
:100B6D000250027A027892E6FF306002617685517A
:100B7D0092855293D26043E680C3E49AF8E49BF9E0
:100B8D003066028102E8FAE9FBD3E913FDE813FCB4
:100B9D0088518952C3EF94036038EF20E00DE82CA3
:100BAD00F8E93DF9ECFAEDFB020BCBE828F8E93951
:100BBD00F9C3E82402F8E93400F97AFE7BFFC3EFAC
:100BCD009403400E8A538B54884D894E8C4F8D5013
:100BDD008136885389548A4D8B4E8C4F8D50306998
:100BED00127553F07554FF754FF07550FF7551F038
:100BFD007552FF8136E8FAD3E813FC8851C3EF94A0
:100C0D00036020EF20E007E82CF8ECFA8122E828B9
:100C1D002402F87AFEC3EF940340088A53884D8C62
:100C2D004F813688538A4D8C4FE568C3335002642B
:100C3D006BF5683060028140753402D26043E68006
:100C4D00E52D54066034A840A941C3E913F9E81312
:100C5D00F8C3E913F9E813F8306904E92440F9C23F
:0E0C6D00AF53E67F759100C3E498F594E499C7
:100C7B00F595759104D26043E680D2AF22D26475AC
:100C8B004300752000306C03752040020CA7D26422
:100C9B00754300752040306C037520007801790195
:100CAB00206620E52D54066002C2647914E541C329
:100CBB0013700104F8C3941440027814306904785B
:100CCB001B791B206010E543600C306903D534049D
:100CDB00D26DA15A91480543E59E7005E59B020C28
:100CEB00EEE59A5440B52002A14430690908C3E8E7
:100CFB009940011881CE20640A08C3E8994002810B
:100D0B00A781CEC264C2AF53E67F759100306612E5
:100D1B007594007595F8759104D26043E680D2AF57
:100D2B0081A7E5417EFFC3334005C3334001FEC3BA
:100D3B00E49E759400F595A121C3E533940150020F
:100D4B0081A730640281A7D802A15881CEC26DC29F
:100D5B00AF53E67F75910085539485549575910437
:100D6B00854D92854E93D26043E680D2AFE52D54EC
:100D7B00066008206A020533020D96306D0D206C5B
:100D8B000A206407158115810216692278003064E8
:100D9B00027801E53775F007A4F9E5F028F5F0E9DD
:100DAB00A2F013A2F113A2F213F537C394785003F8
:100DBB00753778C3E53795384008D265C293C2952D
:100DCB00C297306002A1CD854F92855093D260437C
:100DDB00E68022207D19C2AF754202C294D29230B6
:100DEB006202D297D2AF759F33759E00020FE0C29D
:100DFB00AF754202C294D296306202D293D2AF75D3
:100E0B009F33759E00020FE0307243207D20C2AFEE
:100E1B0075420390013A757B10C297C296306204FB
:100E2B00D295C131D294D2AF759E23020FE0C2AFDF
:100E3B0075420390013A757B10C293C292306204E3
:100E4B00D295C151D294D2AF759E22020FE0207D74
:100E5B0017C2AF754203900115C297306202D2954B
:100E6B00D2AF759E23020FE0C2AF754203900115FE
:100E7B00C293306202D295D2AF759E22020FE02050
:100E8B007D16C2AF754204C292D296306202D295E1
:100E9B00D2AF759E22020FE0C2AF754204C296D24A
:100EAB0092306202D295D2AF759E23020FE0307260
:100EBB0049207D23C2AF754205900129757B04C281
:100ECB0095C294306204D293C1D7D292D2AF759FA0
:100EDB0033759E00020FE0C2AF75420590014B7552
:100EEB007B40C295C294306204D297C1FAD296D29B
:100EFB00AF759F33759E00020FE0207D1AC2AF7550
:100F0B00420590010BC295306202D293D2AF759F0E
:100F1B0033759E00020FE0C2AF75420590011FC2F0
:100F2B00953062E8D297D2AF759F33759E00020F52
:100F3B00E0207D16C2AF754206C296D29430620293
:100F4B00D293D2AF759E23020FE0C2AF754206C299
:100F5B0092D294306202D297D2AF759E22020FE0EA
:100F6B00307244207D20C2AF75420190014B757BDE
:100F7B0040C293C292306204D297E189D296D2AF2B
:100F8B00759E22020FE0C2AF754201900129757B5D
:100F9B0004C297C296306205D293020FAAD292D2A4
:100FAB00AF759E23020FE0207D17C2AF75420190F3
:100FBB00011FC293306202D297D2AF759E22020FED
:100FCB00E0C2AF75420190010BC297306202D2931F
:100FDB00D2AF759E23C26522900109757B00C29327
:100FEB00C295C297C292C294C296C2622278807690
:100FFB00070876070876010876040876FF0876FF5F
:10100B00087607087602087601087601788C760157
:10101B000876000876B40876FF0876FF0876FF0896
:10102B0076030876FF0876010876FF0876250876A2
:10103B00D00876780876C80876040876FF0876011B
:10104B0008760008767A087610087601087601088B
:10105B0076000876FF087600227887E6FFC272BF1B
:0E106B000302D2727888C27DE630E102D27DA7
:10107900C27E7889E630E102D27EC3EF940260082D
:10108900758E01D273021096758E00C27322788014
:10109900E6149000809378A5F67881E61490008094
:1010A9009378A6F67886E61490008D9378A7F6785B
:1010B9009FE6F87005756B0001DDC3E894114002E5
:1010C9007811E82828F56B256B256B28F56C256BBD
:1010D9002828F56D7886E6F539C3940250037539E9
:1010E90002789CE67538FFB402037538A0B403038F
:1010F90075388278A3E61490009A93F566120FE387
:1011090022227896E6FA7897E6FB7888E6B4030512
:10111900C3EB940EFB307F047A007BFFC3EB9AFC90
:10112900C3948250027C827572000572EC8572F05C
:10113900A4C3E5F0947D40F222D27F310B12055B06
:1011490012055B7A007B007C10120551E55C2AFAD6
:1011590074003BFBDCF37C04C3EB13FBEA13FADCFE
:10116900F7FEC27F310B22757C00757D00E5EF200B
:10117900E6037520000520903DFFE52014600690E8
:101189001FFF1460009304600375EF1653D9BF75F0
:1011990081C043FF8012054C75EF0643B203E5B3E6
:1011A900240220E70DF521E5B120E0068521B343AE
:1011B900B101120FE375800875A40075F1FF75D4AC
:1011C900F775900275A5FC75F2FC75D50075A0FD43
:1011D90075A60275F30275D60075B0FF75A701757E
:1011E900F4FF75E241120FE3E4F8F6D8FD756801E2
:1011F900120FF81216C078988673753001C2AF12B3
:10120900056512057512055B12057C12055B120551
:101219008312055B1217F312056512056512056045
:10122900C2AF757C00757D0078FA79FA308307D9E9
:10123900FBD8F7021C0011641197310A310B789819
:101249008673120FE375881075890275C824759124
:101259000475D84075A82275B80275E690759B800B
:10126900759D00759A80759C0075D10E75BC587571
:10127900BB0175BA1F75E88012054CD2AF1208A4DC
:1012890075360053DACF207E0343DA20307E0343DC
:10129900DA1043DA01C2D8C271120565D2617B0343
:1012A9007A0CE55B70077A0CDB0302122912055BE5
:1012B900207003021229C270E55CC3940240E1E583
:1012C9002F541F855E5DF55EB55DD5DAD5C26153D4
:1012D900DACF207E0343DA20307E0343DA10C2D806
:1012E900C27178A2E67008D274E52F54E0F52FC2D6
:1012F90075752900120560307409C3E529940A40FF
:1013090002D27512055178023074027800C3E55C87
:101319009840F0C2AF120575120575120575D2AF66
:10132900120565754C00120551788CE6C39401507D
:101339000302141CE530C39401500302141C757C8C
:10134900A5757DF1207435C3E55C94FF5003021443
:101359001CC2AF12058AD2AF120560C3E55C9401C5
:1013690050EFC2AF120575120556120575D2AF12AC
:101379000560C3E55C94FF40E90218787F05D27FD8
:10138900310B120560C2AFC27F310BAE5CC3E55CA5
:10139900947FD2AF5002812C12054CC2AF12058A3C
:1013A900D2AFDFDA3142C3EE94057897F6120565BC
:1013B9001217FB7F0AD27F310B120560C2AFC27FC1
:1013C900310BAE5CC3E55C947FD2AF50E612054C9D
:1013D900C2AF120575120556120575D2AFDFD631A7
:1013E90042EE24037896F6F87997E7C3948240038E
:1013F900985006E824827897F612056512170E129E
:10140900182A120560310BC3E55C94FF500261474D
:10141900021878757C00757D00C3E55C954C400326
:10142900855C4C12056078017988E7B40302780578
:10143900C3E55C984002612FC2AF12058A12058A82
:1014490012058AD2AF120565753000E4F531F5321F
:101459000531E531F4703F0532789AE67819146060
:0E14690012783214600D787D14600878FA1441
:101477006003753200C3E53298401D120FE3120571
:101487004C153275310078998673C2AF12058AD22E
:10149700AF78988673120560120556E52A700530F5
:1014A7007402412978012074027806C3E55C9840EC
:1014B700A1120560E52A7003021229C2AF120FE3D9
:1014C700E4F522F523F524F525F526F567D2AF785F
:1014D70085E6C333F565E4F544F545F546F547F587
:1014E70048F570F52CF52DF53775700875BB1E128C
:1014F700054C12093530EDFDA8BDA9BEE97001F80C
:10150700887112093975700875BB1E1164C2AF75F1
:1015170061FF1209F2852261852262852263D2AFBB
:101527007522017524017525017526018560697588
:101537006A017888E6B40307C27D307602D27DD28D
:1015470068D269753300120F3C120F6B120A121220
:101557000A19120A12120A19120A12120C99120601
:101567006B120D97120DDE120A19120C88306E03DA
:1015770012070B20660312085E30660312088E12EC
:101587000D97120E13120A19120C99306E031207D7
:1015970047120D97120E8A120A19120C88306E0321
:1015A7001207A5120D97120EB9120A19120C9930CB
:1015B7006E03120802120D97120F3C120A19120934
:1015C70035120C88120D97120F6B120939120A196E
:1015D70030692C856461856462856069756A017903
:1015E700187A0CC3E533994009C269D26A8A350271
:1015F7001606C3E55C9401400302156202167130BA
:101607006A25206C22E535147006C26AD26BA16286
:10161700F535C3E55C940140030215627888E6C39B
:1016270094036003021671753600C3E55F940140A9
:1016370009856462856069756A0178FA79A4E7604B
:10164700027803C3E55F985021307404E52A601AD5
:1016570078F0306C058564617820C3E541985002C5
:10166700A1620536E55C6002C174753600C2AF122F
:101677000FE37887E6FE760211647887EEF6E4F5E5
:1016870022F523F524F525F526F565752C00752D2E
:1016970000D2AF120560120FE378A4E66006D2937A
:1016A700D295D297307406E52A70024129788DE6E3
:1016B700C394014002610C8154901A0D78201217CF
:1016C70050E520B4A50CA3121750E520B45A030225
:1016D70016EE757CA5757DF1120FF812170E757C45
:1016E70000757D0002170D901A0378807B0A121788
:1016F70050A308DBF9901A0F788C7B19121750A3A7
:1017070008DBF9901A2822C2AF12179312177090AC
:101717001A00740E121755A37409121755A37415DE
:10172700121755901A0378807B0A121754A308DB07
:10173700F9901A0F788C7B19121754A308DBF9124A
:1017470017A6121784901A2822E493F622E6438FED
:1017570001538FFDFFC3E583941C400122EF857C75
:10176700B7857DB7F0538FFE22438F02438F0185E4
:101777007CB7857DB7901A0DF0538FFC22901A0D18
:1017870074A5F155901A0E745AF155227A3079D012
:101797007820901A40F150E520F709A3DAF7227A6A
:1017A7003079D0901A40E7F15509A3DAF922AB74E2
:1017B700A875BB01027980BB02027981BB0302795C
:1017C70082BB04027994BB05027983BB0602798642
:1017D700BB07027992BB08027987BB0902799CBBD8
:1017E7000A027988BB0B027989E8F7227C05120582
:1017F70065DCFB22C2AF12057512057C1205831248
:10180700058A12055612057512057C120583120505
:101817008A12055612057512057C12058312058A70
:10182700D2AF22C2AF12058A12058312057C1205B8
:101837007512055612058A12058312057C12057565
:1018470012055612058A12058312057C120575D2F8
:10185700AF22AE74AF75C2AF1205751205751205CA
:0E18670075120556DEF212058A120556DFF8DC
:10187500D2AF221217FB1217F31217F37574017505
:10188500750175760011597C05AD5C120565C3EDD2
:10189500955C70F5C3E55C9401400AC3E55C94FF73
:1018A50040370218BB1217B512170E1217FBC2AF3D
:1018B50075EF161217F3DCD10576C3E57694035060
:1018C5000280C21217F30575E5741490009F93F812
:1018D50008C3E57598500280A91217F31217F3058E
:1018E50074C3E574940C50028095120FF812170E0C
:0818F500C2AF75EF161217F3E4
:0319FD0002117064
:101A00000E091507070104FFFF07020101A55A018E
:101A100000B4FFFFFF03FF01FF25D078C804FF01DA
:091A200000FF10010100FF00FFAE
:101A400023506C6174696E756D31353041232020EF
:101A500023424C48454C4923463331302320202033
:101A60002020202020202020202020202020202076
:101C0000C2AFC2D353D9BF7581C043B20343FF8073
:101C1000752438752503B1DC7529A5752AF175E29F
:101C20004043F10853A4F775D4FFD2837DFA7803BB
:101C300079E67C10752200752300901DE97B0675FE
:101C400024987525013083028145208308D8FBD96B
:101C5000F9DCF781B7308308D8FBD9F9DCF781B715
:101C6000B19CE493A3C39A6004DDC381B7DBDBB10D
:101C70008E6002812E7B08E493FAA3B16FDBF87AC1
:101C800030B16F752200752300B18EEAFCEBFDC305
:101C9000ED94FE400EB18E8A278B28ED30E0048A49
:101CA000828B83B18E7AC270D8C3ED94FE601950D6
:101CB000CEBD002BEC600F7520007521FF7529004B
:101CC000752A000200008100A827A9280809D80465
:101CD000D90281DCB192EA89AAF281CE0D81A3C337
:101CE000ED94035053EDA2E092007AC5C3E58294CF
:101CF00000E583941C508A200010438F02438F011B
:101D00008529B7852AB7F0300029A827A92808090E
:101D1000438F01538FFDD804D902A133C3E58394C7
:101D20001C4003A3A11689AAE28529B7852AB7F02A
:101D3000A3A116538FFC817F7AC1BD030CE493A34A
:101D4000FAB153DCF8B14B817F8181AA22AB23B178
:101D50006FEBFAEA6222752608C3E52313F523E543
:101D60002213F52250066323A0632201D526EAB18F
:101D7000DCB1DC75260AEAF4200102D283300102CC
:101D8000C283B1DCC3134002C201D526EB22B1925B
:101D9000EAFB208302A192308302A197752608AE48
:101DA00024AF25C3EF13FFEE13FEB1E0B1DCC3EAAD
:101DB000133083024480FA30E703632201C3E52332
:101DC00013F523E52213F52250066323A0632201B5
:101DD000D526D9E52265236523F52222AE24AF2539
:101DE0000E0FDEFEDFFCD20122424C48656C6934E6
:071DF000373164F310060116
:00000001FF
